:1000000000308A00F9290000831A0A288E00030EA6
:100010008F000F2883128E00030E8F008F148E0E18
:10002000040890000C0891000D08920083128B1EAA
:100030001B280B1978291008840011088C0012085D
:100040008D000F0E830083120E0E8F188316090089
:100050000A108A100A11033E020703188A0A820056
:10006000AA34C034B634C034BB344034DD34C03478
:10007000BA34C034D734C034BB34C034BF34403455
:10008000BF34C034EF340034E8340034DB34C034DF
:10009000B7344034F8340034DD344034EA34C0340A
:1000A000BD34C034BD344034EB344034EB34C03460
:1000B000D634C034DA34C034DB344034D534C034C0
:1000C000DE34C034DF344034ED34C034D534403411
:1000D000D7344034EE34C034BE34C034DF34C0349E
:1000E00080340034FF348034AF348034FA348034C8
:1000F000ED348034B5344034AE34C034BF34803451
:10010000FB340034F7340034B7348034EF348034B7
:10011000EA340034D4340034AE340034D73480347C
:10012000B7340034BD340034ED340034FF340034CF
:10013000BB348034AD348034B5348034D63480342C
:10014000D5348034DB348034F5340034DE3480340C
:10015000F6348034AA340034EB348034AB34C03409
:10016000AF344034FA340034EB340034AD3400346E
:10017000B5340034EE340034DB340034FD34003464
:10018000AA348034FE340034FE348034BE348034EB
:10019000D7340034BB340034DD340034AB340034A5
:1001A000D5340034EE348034AF340034DE340034DF
:1001B000DA340034AB348034DA348034AE34803412
:1001C000BA348034BD348034AB344034FB348034B2
:1001D000F7348034FD348034AF34C034B6348034E6
:1001E000B734C034B0340034BE340034BC340034CE
:1001F000B4340034C0340034F4340034B634003441
:10020000AC340034D0340034F5348034BF3400349E
:10021000D8340034EC340034F0340034E0340034AA
:10022000FC340034DF348034A8340034B834003473
:10023000A0340034DC340034F6340034D6340034D6
:10024000DF340034BA340034EA348034AD34C0349E
:10025000DD348034AD344034B534C034ED34403412
:100260000A148A100A1182071834183419341B34FE
:100270001D341E3421342334253428342A342C34BC
:100280002F3431343434363438343B343D34403414
:10029000423444344634483449344B344C344D347D
:1002A0004E344F344F344F340A148A100A118207E7
:1002B0005C345C3459345834563452344E344934F6
:1002C00043343D3435342E342634203416340D3442
:1002D0000534173420342834313439343E3444342E
:1002E00049344D345234543458345A345B345C34C9
:1002F0000000000027308100170898006430990042
:1003000018089902003065008515980B852985111C
:10031000990B8829083065009B0A20301B02031CBA
:1003200093291C149B01061AA929861DA0291F3098
:100330001A020318A0299A0A1A0830219700A8293E
:100340009A080319A8291A089A031A083021970055
:10035000BB291C1AAD291C169A011A0854219700B2
:100360001F301A020318BB299A0A13301A02031D00
:10037000BB29043086060B118A111B281C1CC629B8
:100380009C19C429083086061C101C1500348030C6
:100390001F02031CCE299C10D929D9291F089400BB
:1003A0001F0894071408282093009C1495019C159D
:1003B0001C174A2A1C111C139C191C179C11931BF7
:1003C0009C159C1AE7299C161C129C191C16950A50
:1003D0000310930D1C1BEE299C1D9C100830150268
:1003E000031CF729940A14082820930095019C12F5
:1003F0004E2A840183012730810001308C008C1D3E
:10040000092A07308101813084000008C0390F3883
:1004100080006400813084000008C0390C04800032
:100420008B168B1781308400801385018601003084
:100430006500103066001C109C101C119C11950169
:100440000F309A001C133230970064009E01503028
:100450001E020318352A9C111C121C111C19332A68
:100460006400BE212E2A9E0A272A9E0120309D006C
:100470001D0A0319552A40301E020318552A1E086A
:10048000890083160814831208089D009E0A1D081F
:100490009F00C7299C1C542A6400DA291C19532A7E
:0E04A0006400BE214E2A4A2A382A252A63000B
:02400E00FD3F74
:104200000A000D0076007600760020007600760029
:1042100076002000760076007600200044004500FD
:10422000200063007400200063007400200063001D
:1042300074002000630074002000630074002000FC
:1042400063007400200063007400200044004E00EE
:104250003400300061006F002000740075007200AF
:104260006E0065007200400075007300730063000B
:0C4270002E0063006F006D002000FF00B6
:00000001FF
